:0200000480007A
:100000006F00C0006F20802C6F20402C93000000F8
:10001000130100009301000013020000930200008E
:100020001303000093030000130400009304000076
:10003000130500009305000013060000930600005E
:100040001307000093070000130800009308000046
:100050001309000093090000130A0000930A00002E
:10006000130B0000930B0000130C0000930C000016
:10007000130D0000930D0000130E0000930E0000FE
:10008000130F0000930F000097020000938202F804
:100090007390523017A100001301C1E4F32240F124
:1000A0009392C2003301510073100134EF20900B82
:1000B000173500001305858B6F20006B8332851088
:1000C000739012148330850003310501833185015B
:1000D000033205028332850203330503833385032C
:1000E000033405048334850483358505033605060A
:1000F00083368506033705078337850703380508E8
:10010000833885080339050983398509033A050AC7
:10011000833A850A033B050B833B850B033C050CA7
:10012000833C850C033D050D833D850D033E050E87
:10013000833E850E033F050F833F850F033505057D
:10014000730020107311011423341100233C31007B
:10015000233041022334510223386102233C7102CF
:1001600023308104233491042338A104233CB104B7
:100170002330C1062334D1062338E106233CF1069F
:10018000233001092334110923382109233C310983
:100190002330410B2334510B2338610B233C710B6B
:1001A0002330810D2334910D2338A10D233CB10D53
:1001B0002330C10F2334D10F2338E10F233CF10F3B
:1001C000F312011423385100F32200102330511090
:1001D000F322101423345110F32230142338511019
:1001E000F3222014233C5110130501006F208033AB
:1010000000000000000000000000000000000000E0
:1010100000000000000000000000000000000000D0
:1010200000000000000000000000000000000000C0
:1010300000000000000000000000000000000000B0
:081040000000000000000000A8
:10200000B367B500B3E7C70093F77700B306C50021
:10201000638407023386C50093070500637ED502FB
:1020200003C705009385150093871700A38FE7FE6C
:10203000E398C5FE67800000E37ED5FE93070500A8
:1020400003B70500938787009385850023BCE7FECF
:10205000E3E8D7FE6780000067800000130101FFFE
:10206000B367C500233081002334110093F7770054
:10207000130405003307C500638207026376E50099
:1020800093F5F50FEFF09FFD8330810013050400F9
:1020900003340100130101016780000093F5F50F7F
:1020A00093968500B3E6B60093970601B3E7D70091
:1020B00093960702B3E6F600E378E5FC9307050084
:1020C0009387870023BCD7FEE3ECE7FE83308100D3
:1020D00013050400033401001301010167800000AF
:1020E00083470500638E07009307050003C71700A9
:1020F00093871700E31C07FE3385A7406780000025
:1021000013050000678000008347050093851500D4
:102110001305150003C7F5FF638A0700E386E7FE92
:102120001B8507003B05E5406780000013050000A4
:102130006FF05FFFB367B50093F77700639E070208
:10214000137886FF330805016378050393070500BC
:102150006F000001938787009385850063F807016E
:1021600083B6070003B70500E386E6FE3385A74084
:102170003306A640138507003386C5006F00400173
:1021800003C705008347F5FF93851500639AE700B1
:1021900013051500E396C5FE1305000067800000D7
:1021A0003B85E740678000009307050003C70500F3
:1021B0009387170093851500A38FE7FEE31807FEAA
:1021C000678000000347050093060002930705009F
:1021D0006318D70003C7170093871700E30CD7FED7
:1021E0009306D0026300D7069306B0026300D704BB
:1021F00083C60700930500006382060413050000F0
:1022000093871700131725001B8606FD83C607005A
:102210003307A700131717003305E600E39206FE05
:10222000638005023305A0406780000083C6170065
:102230009305000093871700E39206FC1305000046
:102240006780000083C6170093051000938717006E
:10225000E39606FA130500006FF09FFE8347050022
:10226000638007049305101017F7FFFF130787D942
:10227000939505030336070013051500B3E6B70071
:10228000630A060097F7FFFF23BE07DA83370700CC
:10229000E39A07FE2330D70083470500E39C07FC41
:1022A0006780000017F7FFFF1307C7D583370700C4
:1022B000638A070097F7FFFF23B607D88337070025
:1022C000E39A07FE2330A7006F000000130101FF0F
:1022D0001305903423341100EFF0DFFC130101FEED
:1022E0001306810093077101130890006F008000AE
:1022F000930707009376F500138706009305000304
:102300006374D800930570053B07B7002380E7008E
:10231000135545001387F7FFE31CF6FC8347810044
:10232000230C0100638207041305101093060600B6
:1023300017F7FFFF130707CD1315050383350700B4
:102340009386160033E6A700638A050097F7FFFF20
:1023500023BA07CE83370700E39A07FE83C7060038
:102360002330C700E39C07FC1301010267800000D3
:10237000130101FF37F8FFFF233411003307050174
:10238000B7E703006378F7141357C5009306076097
:1023900017360000130606C793973600B307F600FA
:1023A00083B70700337505016390070E977500002A
:1023B0009385C5C503B805006302081483378800F8
:1023C0009778000083B808C423B0F500638E170F18
:1023D0008337080093983600B308160193D7C700D7
:1023E0009397A70013E3F70D93E5F70123B0680077
:1023F00073000512972700009387C7C01317470083
:10240000B387E70003B7070063140710033708001A
:10241000B708040023B0E7000337880023B4E700BF
:10242000F3A80810B707E0FFB307F500371800005E
:10243000130705003388070103BF070083BE870029
:1024400003BE070103B387012330E7012334D7011B
:102450002338C701233C670093870702130707024D
:10246000E39C07FD7390081093973600B306F600BF
:1024700023B0B600730005120F10000083308100F6
:10248000130101016780000013F70704630A0702C4
:1024900013F70708631A07041307F00093E7070808
:1024A0006394E50493963600B306D60023B0F60095
:1024B0007300051283308100130101016780000061
:1024C00093E707046FF01FFE9777000023BC07B265
:1024D0006FF01FF017150000130545ADEFF01FD882
:1024E00013053000EFF01FDC17150000130585B051
:1024F000EFF0DFD613053000EFF0DFDA171500003C
:102500001305C5B3EFF09FD513053000EFF09FD949
:1025100017150000130505B4EFF05FD41305300064
:10252000EFF05FD883358511130101F82338810658
:10253000233C11062334910623302107233C310527
:10254000233841052334510523306105233C7103B1
:1025500023388103233491032330A103233CB101A9
:102560009307800013040500638AF50E930720008B
:102570006380F506938745FF130710006376F70025
:102580009307F0006392F51A03350411EFF05FDE54
:102590001305040003340107833081078334810667
:1025A0000339010683398105033A0105833A810421
:1025B000033B0104833B8103033C0103833C810211
:1025C000033D0102833D8101130101086FD01FAF5C
:1025D000033785109377370063980706EF0780006D
:1025E000731030000327070083A70700630AF7046E
:1025F000130510109307100497160000938686A900
:1026000017F7FFFF130707A013150503833507000E
:102610009386160033E6A700638A050097F7FFFF4D
:1026200023B207A283370700E39A07FE83C7060099
:102630002330C700E39C07FC13053000EFF09FC672
:1026400013051000EFF01FC617150000130585AE27
:10265000EFF0DFC013053000EFF0DFC403290505FC
:10266000371C0000972400009384C499973B000016
:10267000938B4B99370B0400B70AE0FF977D00005E
:10268000938D4D98177A0000130A4A98B7F9030002
:102690006F0080012334F70023B0FD00B71700005E
:1026A000330CFC00630E3C0B9357CC001394470093
:1026B0003387840003370700E30207FE9387076030
:1026C00093973700B387FB0083BC070093F70C0494
:1026D000638E0706732D0B1037160000B3055C01DF
:1026E00013050C002334B100EFF0DFA4630E0500E6
:1026F00093FC0C088335810063800C0437160000BE
:1027000013050C00EFF0DF8FB387840073100D10FA
:1027100003B70D0023B00700E31E07F623B0FD004A
:102720002330FA006FF09FF717150000130505A37B
:10273000EFF0DFB26FF05FF0171500001305059C96
:10274000EFF0DFB113053000EFF0DFB51715000033
:1027500013054597EFF09FB013053000EFF09FB4DD
:1027600013050900EFF01FB4F32740F1639A07182F
:102770009757000093870789130101ED93D7C7008E
:1027800023308112176800001308C887130405005E
:102790009397A700174500001305C586233411122F
:1027A0009356C5001357C80093E7170097380000E9
:1027B000938848851306F0FF233CF5FE9396A60008
:1027C0001317A700B707002093E61600136717003A
:1027D00093D5C8001313F6039387F70C233CF8FE38
:1027E00023B0D8002330E500B3E7650073900718E5
:1027F00073270018639EE7141356B6009307F00181
:102800009702000093824201F39252307310063B0C
:102810007390073A739052301308F0BF13185801A1
:1028200097E7FFFF93874792B3870701739057108D
:10283000F3270034B387070173900714B7B700007C
:102840009B87071073902730B7E701009B870760CD
:10285000739007307350403017270000130787B973
:102860009307083EB3060701B307F700B70808004F
:1028700017660000233CD67817230000130383F665
:102880009766000023B0F6789388F80393078000DA
:102890001308080113D61700B3861701B347F600D3
:1028A000B30507019396C600939757002330D700CE
:1028B0002334B70093F7070213070701B367F60045
:1028C000E31AE3FC13060012930500001305010050
:1028D0009727000023B407F0EFF04FF8B707008008
:1028E0003304F4001305010023348110EFD00FFDF1
:1028F0008330811203340112130101136780000039
:1029000013071000B7779806370608009387F7D1AA
:102910001306C6FF1315F7019316E7036F00C001F6
:102920002F20070013D71700B3C7E7009397E703DB
:10293000B3F7D700B3E7E70033F7C70093F5170005
:102940003307A700E39E05FC032007006FF09FFDFF
:102950001715000013058583EFF05F901305300015
:10296000EFF05F9467800000B70000801301000063
:102970003BD72000B70300809301200063187760E5
:10298000B7000080130110003BD72000B7030040C0
:1029900093013000631C775EB70000801301700064
:1029A0003BD72000B7030001930140006310775E1E
:1029B000B70000801301E0003BD72000B7030200FE
:1029C000930150006314775CB70000809B80100077
:1029D0001301F0013BD72000930310009301600026
:1029E0006316775A9300F0FF130100003BD72000D5
:1029F0009303F0FF93017000631A77589300F0FF80
:102A0000130110003BD72000B70300809B83F3FF26
:102A100093018000631C77569300F0FF1301700050
:102A20003BD72000B70300029B83F3FF9301900084
:102A3000631E77549300F0FF1301E0003BD72000A2
:102A4000B70304009B83F3FF9301A0006310775446
:102A50009300F0FF1301F0013BD720009303100017
:102A60009301B00063147752B72021219B8010128C
:102A7000130100003BD72000B72321219B831312B1
:102A80009301C00063147750B72021219B8010125E
:102A9000130110003BD72000B79390109B830309CC
:102AA0009301D0006314774EB72021219B80101230
:102AB000130170003BD72000B74342009B832324BF
:102AC0009301E0006314774CB72021219B80101202
:102AD0001301E0003BD72000B78300009B834348ED
:102AE0009301F0006314774AB72021219B801012D4
:102AF0001301F0013BD72000930300009301000174
:102B000063167748B72021219B801012130100FE25
:102B10003BD72000B72321219B831312930110017F
:102B200063167746B72021219B801012130110FEF7
:102B30003BD72000B79390109B830309930120019A
:102B400063167744B72021219B801012130170FE79
:102B50003BD72000B74342009B83232493013001DD
:102B600063167742B72021219B8010121301E0FEEB
:102B70003BD72000B78300009B834348930140016B
:102B800063167740B72021219B8010121301F0FFBC
:102B90003BD7200093030000930150016318773E58
:102BA000B720F1FF9B8050349390C00093808067E2
:102BB000130100003BD72000B75334129B83836777
:102BC0009301C0026314773CB720F1FF9B8050341F
:102BD0009390C00093808067130140003BD7200092
:102BE000B74323019B8373569301D0026310773A56
:102BF000B72009009B8050349390C0009380806779
:102C0000130100003BD72000B75334929B838367A6
:102C10009301E002631C7736B72009009B80503493
:102C20009390C00093808067130140003BD7200041
:102C3000B74323099B8373569301F00263187734DB
:102C4000B700008013017000BBD02000B703000163
:102C500093016001639C7032B70000801301E000B3
:102C60003BD12000B7030200930170016310713261
:102C700093007000BBD0100093030000930180010B
:102C80006396703013020000B700008013017000DB
:102C90003BD7200013030700130212009302200009
:102CA000E31452FEB7030001930190016310732EE9
:102CB00013020000B70000801301E0003BD72000A2
:102CC00013000000130307001302120093022000F8
:102CD000E31252FEB70302009301A0016318732AA6
:102CE00013020000B70000801301F0013BD7200061
:102CF000130000001300000013030700130212006A
:102D000093022000E31052FE930310009301B001E0
:102D1000631E732613020000B700008013017000C9
:102D20003BD720001302120093022000E31652FE4C
:102D3000B70300019301C001631A77241302000056
:102D4000B70000801301E000130000003BD7200013
:102D50001302120093022000E31452FEB703020094
:102D60009301D0016314772213020000B7000080A2
:102D70001301F00113000000130000003BD72000F6
:102D80001302120093022000E31252FE930310007C
:102D90009301E001631C771E13020000B70000805E
:102DA00013000000130170003BD720001302120033
:102DB00093022000E31452FEB70300019301F001D7
:102DC0006316771C13020000B70000801300000098
:102DD0001301E000130000003BD720001302120093
:102DE00093022000E31252FEB70302009301000297
:102DF000631E771813020000B70000801300000064
:102E0000130000001301F0013BD720001302120051
:102E100093022000E31252FE93031000930110026C
:102E2000631677161302000013017000B7000080CC
:102E30003BD720001302120093022000E31652FE3B
:102E4000B7030001930120026312771413020000FC
:102E50001301E000B7000080130000003BD7200002
:102E60001302120093022000E31452FEB703020083
:102E700093013002631C7710130200001301F0016C
:102E8000B700008013000000130000003BD72000B3
:102E90001302120093022000E31252FE930310006B
:102EA000930140026314770E1302000013017000B7
:102EB00013000000B70000803BD72000130212006F
:102EC00093022000E31452FEB70300019301500265
:102ED000631E770A130200001301E00013000000D4
:102EE000B7000080130000003BD72000130212003F
:102EF00093022000E31252FEB70302009301600226
:102F000063167708130200001301F001130000009C
:102F100013000000B70000803BD72000130212000E
:102F200093022000E31252FE9303100093017002FB
:102F3000631E77049300F0003B51100093030000E0
:102F40009301800263147104930000023BD10000DE
:102F50009303000293019002631A7102BB500000B8
:102F6000930300009301A00263927002930000405B
:102F7000371100001B0101803BD0200093030000AB
:102F80009301B00263147000631A300013951100AE
:102F900063000500136515007300000013051000A1
:082FA00073000000731000C073
:102FA800417373657274696F6E206661696C6564DC
:102FB8003A2061646472203E3D202831554C203C03
:102FC8003C203132292026262061646472203C206E
:102FD8003633202A202831554C203C3C20313229D8
:102FE8000A00000000000000417373657274696F85
:102FF8006E206661696C65643A20212870745B33C1
:103008005D5B616464722F2831554C203C3C203153
:1030180032295D2026203078303830292026262095
:103028006361757365203D3D203078660A000000B5
:10303800417373657274696F6E206661696C65644B
:103048003A206E6F64650A00417373657274696F24
:103058006E206661696C65643A20757365725F6D90
:10306800617070696E675B616464722F2831554CBA
:10307800203C3C203132295D2E61646472203D3D44
:1030880020300A0000000000417373657274696F94
:103098006E206661696C65643A202122696C6C65F2
:1030A80067616C20696E737472756374696F6E22E0
:1030B8000A00000000000000417373657274696FB4
:1030C8006E206661696C65643A2070745B335D5B81
:1030D800616464722F2831554C203C3C20313229E0
:1030E8005D20262030783034300A000000000000CF
:1030F800417373657274696F6E206661696C65648B
:103108003A2070745B335D5B616464722F283155BB
:103118004C203C3C203132295D2026203078303844
:10312800300A000000000000417373657274696F13
:103138006E206661696C65643A2074662D3E657020
:103148006320252034203D3D20300A000000000087
:10315800417373657274696F6E206661696C65642A
:103168003A202122756E6578706563746564206500
:103178007863657074696F6E220A000000000000B1
:10318800417373657274696F6E206661696C6564FA
:103198003A202122756E737570706F7274656420A1
:0C31A80073617470206D6F6465220A0072
:040000058000000077
:00000001FF
